 redefclass028

 Timestamp is 86d5f8ab (reproducible build file hash)

 Preferred load address is 0000000180000000

 Start         Length     Name                   Class
 0001:00000000 00003a80H .text$mn                CODE
 0001:00003a80 00000036H .text$mn$00             CODE
 0001:00003ab6 00000092H .text$x                 CODE
 0002:00000000 000001d0H .idata$5                DATA
 0002:000001d0 00000038H .00cfg                  DATA
 0002:00000208 00000008H .CRT$XCA                DATA
 0002:00000210 00000008H .CRT$XCZ                DATA
 0002:00000218 00000008H .CRT$XIA                DATA
 0002:00000220 00000008H .CRT$XIC                DATA
 0002:00000228 00000008H .CRT$XIZ                DATA
 0002:00000230 00000008H .CRT$XLA                DATA
 0002:00000238 00000008H .CRT$XLZ                DATA
 0002:00000240 00000008H .CRT$XPA                DATA
 0002:00000248 00000008H .CRT$XPZ                DATA
 0002:00000250 00000008H .CRT$XTA                DATA
 0002:00000258 00000008H .CRT$XTZ                DATA
 0002:00000260 00000000H .gehcont$y              DATA
 0002:00000260 00000000H .gfids$y                DATA
 0002:00000260 000024a0H .rdata                  DATA
 0002:00002700 00000000H .rdata$CastGuardVftablesA DATA
 0002:00002700 00000000H .rdata$CastGuardVftablesC DATA
 0002:00002700 00000028H .rdata$T                DATA
 0002:00002728 000000d4H .rdata$voltmd           DATA
 0002:000027fc 0000031cH .rdata$zzzdbg           DATA
 0002:00002b18 00000008H .rtc$IAA                DATA
 0002:00002b20 00000008H .rtc$IZZ                DATA
 0002:00002b28 00000008H .rtc$TAA                DATA
 0002:00002b30 00000008H .rtc$TZZ                DATA
 0002:00002b38 00000004H .tls                    DATA
 0002:00002b3c 00000004H .tls$                   DATA
 0002:00002b40 00000008H .tls$ZZZ                DATA
 0002:00002b48 00000388H .xdata                  DATA
 0002:00002ed0 00000464H .edata                  DATA
 0002:00003334 0000008cH .idata$2                DATA
 0002:000033c0 00000018H .idata$3                DATA
 0002:000033d8 000001d0H .idata$4                DATA
 0002:000035a8 0000048eH .idata$6                DATA
 0003:00000000 00000090H .data                   DATA
 0003:00000090 0001b258H .bss                    DATA
 0004:00000000 00000408H .pdata                  DATA

  Address         Publics by Value              Rva+Base               Lib:Object

 0000:00000000       __AbsoluteZero             0000000000000000     <absolute>
 0000:00000000       ___safe_se_handler_count   0000000000000000     <absolute>
 0000:00000000       ___safe_se_handler_table   0000000000000000     <absolute>
 0000:00000000       __arm64x_extra_rfe_table   0000000000000000     <absolute>
 0000:00000000       __arm64x_extra_rfe_table_size 0000000000000000     <absolute>
 0000:00000000       __arm64x_native_entrypoint 0000000000000000     <absolute>
 0000:00000000       __arm64x_redirection_metadata 0000000000000000     <absolute>
 0000:00000000       __arm64x_redirection_metadata_count 0000000000000000     <absolute>
 0000:00000000       __dynamic_value_reloc_table 0000000000000000     <absolute>
 0000:00000000       __enclave_config           0000000000000000     <absolute>
 0000:00000000       __guard_check_icall_a64n_fptr 0000000000000000     <absolute>
 0000:00000000       __guard_eh_cont_count      0000000000000000     <absolute>
 0000:00000000       __guard_eh_cont_table      0000000000000000     <absolute>
 0000:00000000       __guard_fids_count         0000000000000000     <absolute>
 0000:00000000       __guard_fids_table         0000000000000000     <absolute>
 0000:00000000       __guard_iat_count          0000000000000000     <absolute>
 0000:00000000       __guard_iat_table          0000000000000000     <absolute>
 0000:00000000       __guard_longjmp_count      0000000000000000     <absolute>
 0000:00000000       __guard_longjmp_table      0000000000000000     <absolute>
 0000:00000000       __hybrid_auxiliary_iat     0000000000000000     <absolute>
 0000:00000000       __hybrid_auxiliary_iat_copy 0000000000000000     <absolute>
 0000:00000000       __hybrid_code_map          0000000000000000     <absolute>
 0000:00000000       __hybrid_code_map_count    0000000000000000     <absolute>
 0000:00000000       __x64_code_ranges_to_entry_points 0000000000000000     <absolute>
 0000:00000000       __x64_code_ranges_to_entry_points_count 0000000000000000     <absolute>
 0000:00000100       __guard_flags              0000000000000100     <absolute>
 0000:00000000       __ImageBase                0000000180000000     <linker-defined>
 0001:00000000       ?NewObject@JNIEnv_@@QEAAPEAV_jobject@@PEAV_jclass@@PEAU_jmethodID@@ZZ 0000000180001000 f i libredefclass028.obj
 0001:00000028       ?SetEventNotificationMode@_jvmtiEnv@@QEAA?AW4jvmtiError@@W4jvmtiEventMode@@W4jvmtiEvent@@PEAV_jobject@@ZZ 0000000180001028 f i libredefclass028.obj
 0001:00000034       ?TranslateError@@YAPEBDW4jvmtiError@@@Z 0000000180001034 f   libredefclass028.obj
 0001:000002ec       ?nsk_jni_check_exception@@YAHPEAUJNIEnv_@@QEBDH@Z 00000001800012ec f   libredefclass028.obj
 0001:00000430       ?nsk_jni_lverify@@YAHHPEAUJNIEnv_@@HQEBDH1ZZ 0000000180001430 f   libredefclass028.obj
 0001:000004d0       Agent_Initialize           00000001800014d0 f   libredefclass028.obj
 0001:000007cc       Agent_OnAttach             00000001800017cc f   libredefclass028.obj
 0001:000007cc       Agent_OnLoad               00000001800017cc f   libredefclass028.obj
 0001:000007d4       CompiledMethodLoad         00000001800017d4 f   libredefclass028.obj
 0001:00000950       CompiledMethodUnload       0000000180001950 f   libredefclass028.obj
 0001:00000a08       Java_nsk_jvmti_RedefineClasses_redefclass028_isRedefinitionOccurred 0000000180001a08 f   libredefclass028.obj
 0001:00000a38       Java_nsk_jvmti_RedefineClasses_redefclass028_notifyNativeAgent 0000000180001a38 f   libredefclass028.obj
 0001:00000a6c       Java_nsk_jvmti_RedefineClasses_redefclass028_storeClassBytes 0000000180001a6c f   libredefclass028.obj
 0001:00000abc       Java_nsk_jvmti_unit_FollowReferences_FollowRefObjects_addRefToVerify 0000000180001abc f   libredefclass028.obj
 0001:00000c94       Java_nsk_jvmti_unit_FollowReferences_FollowRefObjects_getTag 0000000180001c94 f   libredefclass028.obj
 0001:00000d54       Java_nsk_jvmti_unit_FollowReferences_FollowRefObjects_resetRefsToVerify 0000000180001d54 f   libredefclass028.obj
 0001:00000d5c       Java_nsk_jvmti_unit_FollowReferences_FollowRefObjects_resetTags 0000000180001d5c f   libredefclass028.obj
 0001:00000da0       Java_nsk_jvmti_unit_FollowReferences_FollowRefObjects_setTag 0000000180001da0 f   libredefclass028.obj
 0001:00000ff8       Java_nsk_share_jvmti_ArgumentHandler_getAgentOptionsString 0000000180001ff8 f   libredefclass028.obj
 0001:000010a8       Java_nsk_share_jvmti_DebugeeClass_checkStatus 00000001800020a8 f   libredefclass028.obj
 0001:00001130       Java_nsk_share_jvmti_DebugeeClass_resetAgentData 0000000180002130 f   libredefclass028.obj
 0001:00001190       Java_nsk_share_jvmti_RedefineAgent_agentStatus 0000000180002190 f   libredefclass028.obj
 0001:0000119c       Java_nsk_share_jvmti_RedefineAgent_isRedefined 000000018000219c f   libredefclass028.obj
 0001:000011a8       Java_nsk_share_jvmti_RedefineAgent_redefineAttempted 00000001800021a8 f   libredefclass028.obj
 0001:000011b4       MA_checkStatus             00000001800021b4 f   libredefclass028.obj
 0001:00001258       __local_stdio_printf_options 0000000180002258 f i libredefclass028.obj
 0001:00001960       exitOnError                0000000180002960 f   libredefclass028.obj
 0001:00001a14       fprintf                    0000000180002a14 f i libredefclass028.obj
 0001:00001a58       nsk_complain               0000000180002a58 f   libredefclass028.obj
 0001:00001a84       nsk_jvmti_createJVMTIEnv   0000000180002a84 f   libredefclass028.obj
 0001:00001bb4       nsk_jvmti_enableEvents     0000000180002bb4 f   libredefclass028.obj
 0001:00001c88       nsk_jvmti_lverify          0000000180002c88 f   libredefclass028.obj
 0001:00001d78       nsk_jvmti_parseOptions     0000000180002d78 f   libredefclass028.obj
 0001:00001fc8       nsk_jvmti_resetAgentData   0000000180002fc8 f   libredefclass028.obj
 0001:00002048       nsk_jvmti_resumeSync       0000000180003048 f   libredefclass028.obj
 0001:000020f0       nsk_jvmti_setFailStatus    00000001800030f0 f   libredefclass028.obj
 0001:0000212c       nsk_jvmti_waitForSync      000000018000312c f   libredefclass028.obj
 0001:00002230       nsk_lcomplain              0000000180003230 f   libredefclass028.obj
 0001:00002250       nsk_ldisplay               0000000180003250 f   libredefclass028.obj
 0001:00002270       nsk_ltrace                 0000000180003270 f   libredefclass028.obj
 0001:00002290       nsk_lvcomplain             0000000180003290 f   libredefclass028.obj
 0001:00002448       nsk_lvdisplay              0000000180003448 f   libredefclass028.obj
 0001:00002494       nsk_lverify                0000000180003494 f   libredefclass028.obj
 0001:000024f0       nsk_lvtrace                00000001800034f0 f   libredefclass028.obj
 0001:00002550       nsk_printf                 0000000180003550 f   libredefclass028.obj
 0001:00002578       nsk_vprintf                0000000180003578 f   libredefclass028.obj
 0001:0000262c       printf                     000000018000362c f i libredefclass028.obj
 0001:00002b54       __raise_securityfailure    0000000180003b54 f   MSVCRT:gs_report.obj
 0001:00002b88       __report_gsfailure         0000000180003b88 f   MSVCRT:gs_report.obj
 0001:00002dc8       __GSHandlerCheck           0000000180003dc8 f   MSVCRT:gshandler.obj
 0001:00002de8       __GSHandlerCheckCommon     0000000180003de8 f   MSVCRT:gshandler.obj
 0001:00002e60       __security_check_cookie    0000000180003e60 f   MSVCRT:amdsecgs.obj
 0001:000031a0       _DllMainCRTStartup         00000001800041a0 f   MSVCRT:dll_dllmain.obj
 0001:000031e0       __scrt_acquire_startup_lock 00000001800041e0 f   MSVCRT:utility.obj
 0001:0000321c       __scrt_dllmain_after_initialize_c 000000018000421c f   MSVCRT:utility.obj
 0001:00003250       __scrt_dllmain_before_initialize_c 0000000180004250 f   MSVCRT:utility.obj
 0001:00003268       __scrt_dllmain_crt_thread_attach 0000000180004268 f   MSVCRT:utility.obj
 0001:00003290       __scrt_dllmain_crt_thread_detach 0000000180004290 f   MSVCRT:utility.obj
 0001:000032a8       __scrt_dllmain_exception_filter 00000001800042a8 f   MSVCRT:utility.obj
 0001:00003308       __scrt_dllmain_uninitialize_c 0000000180004308 f   MSVCRT:utility.obj
 0001:00003338       __scrt_dllmain_uninitialize_critical 0000000180004338 f   MSVCRT:utility.obj
 0001:0000334c       __scrt_initialize_crt      000000018000434c f   MSVCRT:utility.obj
 0001:00003398       __scrt_initialize_onexit_tables 0000000180004398 f   MSVCRT:utility.obj
 0001:00003424       __scrt_is_nonwritable_in_current_image 0000000180004424 f   MSVCRT:utility.obj
 0001:000034bc       __scrt_release_startup_lock 00000001800044bc f   MSVCRT:utility.obj
 0001:000034e0       __scrt_uninitialize_crt    00000001800044e0 f   MSVCRT:utility.obj
 0001:0000350c       _onexit                    000000018000450c f   MSVCRT:utility.obj
 0001:00003548       atexit                     0000000180004548 f   MSVCRT:utility.obj
 0001:00003560       __crt_debugger_hook        0000000180004560 f   MSVCRT:utility_desktop.obj
 0001:00003568       __scrt_fastfail            0000000180004568 f   MSVCRT:utility_desktop.obj
 0001:000036b4       _guard_check_icall_nop     00000001800046b4 f i MSVCRT:guard_support.obj
 0001:000036b8       __security_init_cookie     00000001800046b8 f   MSVCRT:gs_support.obj
 0001:00003764       DllMain                    0000000180004764 f   MSVCRT:dll_dllmain_stub.obj
 0001:00003788       ?__scrt_initialize_type_info@@YAXXZ 0000000180004788 f   MSVCRT:tncleanup.obj
 0001:00003798       ?__scrt_uninitialize_type_info@@YAXXZ 0000000180004798 f   MSVCRT:tncleanup.obj
 0001:000037a4       __local_stdio_scanf_options 00000001800047a4 f i MSVCRT:default_local_stdio_options.obj
 0001:000037ac       __scrt_initialize_default_local_stdio_options 00000001800047ac f   MSVCRT:default_local_stdio_options.obj
 0001:000037c8       __scrt_get_dyn_tls_init_callback 00000001800047c8 f   MSVCRT:dyn_tls_init.obj
 0001:000037d0       _RTC_Initialize            00000001800047d0 f   MSVCRT:initsect.obj
 0001:0000380c       _RTC_Terminate             000000018000480c f   MSVCRT:initsect.obj
 0001:00003848       __isa_available_init       0000000180004848 f   MSVCRT:cpu_disp.obj
 0001:000039f4       _get_startup_argv_mode     00000001800049f4 f   MSVCRT:argv_mode.obj
 0001:000039fc       __scrt_is_ucrt_dll_in_use  00000001800049fc f   MSVCRT:ucrt_detection.obj
 0001:00003a10       memcpy                     0000000180004a10 f   vcruntime:VCRUNTIME140.dll
 0001:00003a16       memset                     0000000180004a16 f   vcruntime:VCRUNTIME140.dll
 0001:00003a1c       strchr                     0000000180004a1c f   vcruntime:VCRUNTIME140.dll
 0001:00003a22       __C_specific_handler       0000000180004a22 f   vcruntime:VCRUNTIME140.dll
 0001:00003a28       __std_type_info_destroy_list 0000000180004a28 f   vcruntime:VCRUNTIME140.dll
 0001:00003a2e       strcmp                     0000000180004a2e f   ucrt:api-ms-win-crt-string-l1-1-0.dll
 0001:00003a34       strlen                     0000000180004a34 f   ucrt:api-ms-win-crt-string-l1-1-0.dll
 0001:00003a3a       _initterm                  0000000180004a3a f   ucrt:api-ms-win-crt-runtime-l1-1-0.dll
 0001:00003a40       _initterm_e                0000000180004a40 f   ucrt:api-ms-win-crt-runtime-l1-1-0.dll
 0001:00003a46       _seh_filter_dll            0000000180004a46 f   ucrt:api-ms-win-crt-runtime-l1-1-0.dll
 0001:00003a4c       _configure_narrow_argv     0000000180004a4c f   ucrt:api-ms-win-crt-runtime-l1-1-0.dll
 0001:00003a52       _initialize_narrow_environment 0000000180004a52 f   ucrt:api-ms-win-crt-runtime-l1-1-0.dll
 0001:00003a58       _initialize_onexit_table   0000000180004a58 f   ucrt:api-ms-win-crt-runtime-l1-1-0.dll
 0001:00003a5e       _register_onexit_function  0000000180004a5e f   ucrt:api-ms-win-crt-runtime-l1-1-0.dll
 0001:00003a64       _execute_onexit_table      0000000180004a64 f   ucrt:api-ms-win-crt-runtime-l1-1-0.dll
 0001:00003a6a       _crt_atexit                0000000180004a6a f   ucrt:api-ms-win-crt-runtime-l1-1-0.dll
 0001:00003a70       _cexit                     0000000180004a70 f   ucrt:api-ms-win-crt-runtime-l1-1-0.dll
 0001:00003a78       __acrt_initialize          0000000180004a78 f   MSVCRT:ucrt_stubs.obj
 0001:00003a78       __acrt_thread_attach       0000000180004a78 f   MSVCRT:ucrt_stubs.obj
 0001:00003a78       __acrt_thread_detach       0000000180004a78 f   MSVCRT:ucrt_stubs.obj
 0001:00003a78       __acrt_uninitialize        0000000180004a78 f   MSVCRT:ucrt_stubs.obj
 0001:00003a78       __acrt_uninitialize_critical 0000000180004a78 f   MSVCRT:ucrt_stubs.obj
 0001:00003a78       __scrt_stub_for_acrt_initialize 0000000180004a78 f   MSVCRT:ucrt_stubs.obj
 0001:00003a78       __scrt_stub_for_acrt_thread_attach 0000000180004a78 f   MSVCRT:ucrt_stubs.obj
 0001:00003a78       __scrt_stub_for_acrt_thread_detach 0000000180004a78 f   MSVCRT:ucrt_stubs.obj
 0001:00003a78       __scrt_stub_for_acrt_uninitialize 0000000180004a78 f   MSVCRT:ucrt_stubs.obj
 0001:00003a78       __scrt_stub_for_acrt_uninitialize_critical 0000000180004a78 f   MSVCRT:ucrt_stubs.obj
 0001:00003a78       __vcrt_initialize          0000000180004a78 f   MSVCRT:ucrt_stubs.obj
 0001:00003a78       __vcrt_thread_attach       0000000180004a78 f   MSVCRT:ucrt_stubs.obj
 0001:00003a78       __vcrt_thread_detach       0000000180004a78 f   MSVCRT:ucrt_stubs.obj
 0001:00003a78       __vcrt_uninitialize        0000000180004a78 f   MSVCRT:ucrt_stubs.obj
 0001:00003a78       __vcrt_uninitialize_critical 0000000180004a78 f   MSVCRT:ucrt_stubs.obj
 0001:00003a7c       __scrt_stub_for_is_c_termination_complete 0000000180004a7c f   MSVCRT:ucrt_stubs.obj
 0001:00003a7c       _is_c_termination_complete 0000000180004a7c f   MSVCRT:ucrt_stubs.obj
 0001:00003a90       _guard_dispatch_icall_nop  0000000180004a90 f   MSVCRT:guard_dispatch.obj
 0001:00003ab0       _guard_xfg_dispatch_icall_nop 0000000180004ab0 f   MSVCRT:guard_xfg_dispatch.obj
 0002:00000000       __imp_Sleep                0000000180005000     kernel32:KERNEL32.dll
 0002:00000008       __imp_RtlCaptureContext    0000000180005008     kernel32:KERNEL32.dll
 0002:00000010       __imp_RtlLookupFunctionEntry 0000000180005010     kernel32:KERNEL32.dll
 0002:00000018       __imp_RtlVirtualUnwind     0000000180005018     kernel32:KERNEL32.dll
 0002:00000020       __imp_UnhandledExceptionFilter 0000000180005020     kernel32:KERNEL32.dll
 0002:00000028       __imp_SetUnhandledExceptionFilter 0000000180005028     kernel32:KERNEL32.dll
 0002:00000030       __imp_GetCurrentProcess    0000000180005030     kernel32:KERNEL32.dll
 0002:00000038       __imp_TerminateProcess     0000000180005038     kernel32:KERNEL32.dll
 0002:00000040       __imp_IsProcessorFeaturePresent 0000000180005040     kernel32:KERNEL32.dll
 0002:00000048       __imp_CloseHandle          0000000180005048     kernel32:KERNEL32.dll
 0002:00000050       __imp_InitializeCriticalSectionAndSpinCount 0000000180005050     kernel32:KERNEL32.dll
 0002:00000058       __imp_DeleteCriticalSection 0000000180005058     kernel32:KERNEL32.dll
 0002:00000060       __imp_CreateEventW         0000000180005060     kernel32:KERNEL32.dll
 0002:00000068       __imp_GetModuleHandleW     0000000180005068     kernel32:KERNEL32.dll
 0002:00000070       __imp_GetProcAddress       0000000180005070     kernel32:KERNEL32.dll
 0002:00000078       __imp_IsDebuggerPresent    0000000180005078     kernel32:KERNEL32.dll
 0002:00000080       __imp_QueryPerformanceCounter 0000000180005080     kernel32:KERNEL32.dll
 0002:00000088       __imp_GetCurrentProcessId  0000000180005088     kernel32:KERNEL32.dll
 0002:00000090       __imp_GetCurrentThreadId   0000000180005090     kernel32:KERNEL32.dll
 0002:00000098       __imp_GetSystemTimeAsFileTime 0000000180005098     kernel32:KERNEL32.dll
 0002:000000a0       __imp_DisableThreadLibraryCalls 00000001800050a0     kernel32:KERNEL32.dll
 0002:000000a8       __imp_InitializeSListHead  00000001800050a8     kernel32:KERNEL32.dll
 0002:000000b0       \177KERNEL32_NULL_THUNK_DATA 00000001800050b0     kernel32:KERNEL32.dll
 0002:000000b8       __imp_memcpy               00000001800050b8     vcruntime:VCRUNTIME140.dll
 0002:000000c0       __imp_memset               00000001800050c0     vcruntime:VCRUNTIME140.dll
 0002:000000c8       __imp_strchr               00000001800050c8     vcruntime:VCRUNTIME140.dll
 0002:000000d0       __imp___C_specific_handler 00000001800050d0     vcruntime:VCRUNTIME140.dll
 0002:000000d8       __imp___std_type_info_destroy_list 00000001800050d8     vcruntime:VCRUNTIME140.dll
 0002:000000e0       \177VCRUNTIME140_NULL_THUNK_DATA 00000001800050e0     vcruntime:VCRUNTIME140.dll
 0002:000000e8       __imp_strtol               00000001800050e8     ucrt:api-ms-win-crt-convert-l1-1-0.dll
 0002:000000f0       \177api-ms-win-crt-convert-l1-1-0_NULL_THUNK_DATA 00000001800050f0     ucrt:api-ms-win-crt-convert-l1-1-0.dll
 0002:000000f8       __imp_malloc               00000001800050f8     ucrt:api-ms-win-crt-heap-l1-1-0.dll
 0002:00000100       __imp_free                 0000000180005100     ucrt:api-ms-win-crt-heap-l1-1-0.dll
 0002:00000108       \177api-ms-win-crt-heap-l1-1-0_NULL_THUNK_DATA 0000000180005108     ucrt:api-ms-win-crt-heap-l1-1-0.dll
 0002:00000110       __imp__errno               0000000180005110     ucrt:api-ms-win-crt-runtime-l1-1-0.dll
 0002:00000118       __imp_exit                 0000000180005118     ucrt:api-ms-win-crt-runtime-l1-1-0.dll
 0002:00000120       __imp__cexit               0000000180005120     ucrt:api-ms-win-crt-runtime-l1-1-0.dll
 0002:00000128       __imp__crt_atexit          0000000180005128     ucrt:api-ms-win-crt-runtime-l1-1-0.dll
 0002:00000130       __imp__execute_onexit_table 0000000180005130     ucrt:api-ms-win-crt-runtime-l1-1-0.dll
 0002:00000138       __imp__register_onexit_function 0000000180005138     ucrt:api-ms-win-crt-runtime-l1-1-0.dll
 0002:00000140       __imp__initialize_onexit_table 0000000180005140     ucrt:api-ms-win-crt-runtime-l1-1-0.dll
 0002:00000148       __imp__initialize_narrow_environment 0000000180005148     ucrt:api-ms-win-crt-runtime-l1-1-0.dll
 0002:00000150       __imp__configure_narrow_argv 0000000180005150     ucrt:api-ms-win-crt-runtime-l1-1-0.dll
 0002:00000158       __imp__seh_filter_dll      0000000180005158     ucrt:api-ms-win-crt-runtime-l1-1-0.dll
 0002:00000160       __imp__initterm_e          0000000180005160     ucrt:api-ms-win-crt-runtime-l1-1-0.dll
 0002:00000168       __imp__initterm            0000000180005168     ucrt:api-ms-win-crt-runtime-l1-1-0.dll
 0002:00000170       \177api-ms-win-crt-runtime-l1-1-0_NULL_THUNK_DATA 0000000180005170     ucrt:api-ms-win-crt-runtime-l1-1-0.dll
 0002:00000178       __imp___acrt_iob_func      0000000180005178     ucrt:api-ms-win-crt-stdio-l1-1-0.dll
 0002:00000180       __imp_fflush               0000000180005180     ucrt:api-ms-win-crt-stdio-l1-1-0.dll
 0002:00000188       __imp___stdio_common_vsprintf 0000000180005188     ucrt:api-ms-win-crt-stdio-l1-1-0.dll
 0002:00000190       __imp___stdio_common_vfprintf 0000000180005190     ucrt:api-ms-win-crt-stdio-l1-1-0.dll
 0002:00000198       \177api-ms-win-crt-stdio-l1-1-0_NULL_THUNK_DATA 0000000180005198     ucrt:api-ms-win-crt-stdio-l1-1-0.dll
 0002:000001a0       __imp_strcmp               00000001800051a0     ucrt:api-ms-win-crt-string-l1-1-0.dll
 0002:000001a8       __imp__strdup              00000001800051a8     ucrt:api-ms-win-crt-string-l1-1-0.dll
 0002:000001a8       __imp_strdup               00000001800051a8     ucrt:api-ms-win-crt-string-l1-1-0.dll
 0002:000001b0       __imp_strlen               00000001800051b0     ucrt:api-ms-win-crt-string-l1-1-0.dll
 0002:000001b8       __imp_strpbrk              00000001800051b8     ucrt:api-ms-win-crt-string-l1-1-0.dll
 0002:000001c0       __imp_strncpy              00000001800051c0     ucrt:api-ms-win-crt-string-l1-1-0.dll
 0002:000001c8       \177api-ms-win-crt-string-l1-1-0_NULL_THUNK_DATA 00000001800051c8     ucrt:api-ms-win-crt-string-l1-1-0.dll
 0002:000001d0       __guard_check_icall_fptr   00000001800051d0     MSVCRT:guard_support.obj
 0002:000001d8       __guard_xfg_check_icall_fptr 00000001800051d8     MSVCRT:guard_support.obj
 0002:000001e0       __guard_dispatch_icall_fptr 00000001800051e0     MSVCRT:guard_support.obj
 0002:000001e8       __guard_xfg_dispatch_icall_fptr 00000001800051e8     MSVCRT:guard_support.obj
 0002:000001f0       __guard_xfg_table_dispatch_icall_fptr 00000001800051f0     MSVCRT:guard_support.obj
 0002:000001f8       __castguard_check_failure_os_handled_fptr 00000001800051f8     MSVCRT:guard_support.obj
 0002:00000200       __guard_memcpy_fptr        0000000180005200     vcruntime:softmemtag.obj
 0002:00000208       __xc_a                     0000000180005208     MSVCRT:initializers.obj
 0002:00000210       __xc_z                     0000000180005210     MSVCRT:initializers.obj
 0002:00000218       __xi_a                     0000000180005218     MSVCRT:initializers.obj
 0002:00000228       __xi_z                     0000000180005228     MSVCRT:initializers.obj
 0002:00000230       __xl_a                     0000000180005230     MSVCRT:tlssup.obj
 0002:00000238       __xl_z                     0000000180005238     MSVCRT:tlssup.obj
 0002:00000240       __xp_a                     0000000180005240     MSVCRT:initializers.obj
 0002:00000248       __xp_z                     0000000180005248     MSVCRT:initializers.obj
 0002:00000250       __xt_a                     0000000180005250     MSVCRT:initializers.obj
 0002:00000258       __xt_z                     0000000180005258     MSVCRT:initializers.obj
 0002:00000260       g_refKindStr               0000000180005260     libredefclass028.obj
 0002:00000410       ??_C@_09BPLDFGCI@unknown_0@ 0000000180005410     libredefclass028.obj
 0002:00000420       ??_C@_0BL@FPNMECJD@JVMTI_HEAP_REFERENCE_CLASS@ 0000000180005420     libredefclass028.obj
 0002:00000440       ??_C@_0BL@FKGKKLNM@JVMTI_HEAP_REFERENCE_FIELD@ 0000000180005440     libredefclass028.obj
 0002:00000460       ??_C@_0CD@CAEHCFJF@JVMTI_HEAP_REFERENCE_ARRAY_ELEM@ 0000000180005460     libredefclass028.obj
 0002:00000488       ??_C@_0CC@DNEBMCNK@JVMTI_HEAP_REFERENCE_CLASS_LOAD@ 0000000180005488     libredefclass028.obj
 0002:000004b0       ??_C@_0BN@CJMIPEBB@JVMTI_HEAP_REFERENCE_SIGNERS@ 00000001800054b0     libredefclass028.obj
 0002:000004d0       ??_C@_0CH@HBOIDPEB@JVMTI_HEAP_REFERENCE_PROTECTION@ 00000001800054d0     libredefclass028.obj
 0002:000004f8       ??_C@_0BP@MDKGDGKL@JVMTI_HEAP_REFERENCE_INTERFACE@ 00000001800054f8     libredefclass028.obj
 0002:00000518       ??_C@_0CC@JJMIHNJH@JVMTI_HEAP_REFERENCE_STATIC_FIE@ 0000000180005518     libredefclass028.obj
 0002:00000540       ??_C@_0CD@IDHEEGID@JVMTI_HEAP_REFERENCE_CONSTANT_P@ 0000000180005540     libredefclass028.obj
 0002:00000568       ??_C@_0CA@EFFCHNG@JVMTI_HEAP_REFERENCE_SUPERCLASS@ 0000000180005568     libredefclass028.obj
 0002:00000588       ??_C@_0L@PCDFHGCJ@unknown_11@ 0000000180005588     libredefclass028.obj
 0002:00000598       ??_C@_0L@NJBICFOK@unknown_12@ 0000000180005598     libredefclass028.obj
 0002:000005a8       ??_C@_0L@MAADBEKL@unknown_13@ 00000001800055a8     libredefclass028.obj
 0002:000005b8       ??_C@_0L@IPECICGM@unknown_14@ 00000001800055b8     libredefclass028.obj
 0002:000005c8       ??_C@_0L@JGFJLDCN@unknown_15@ 00000001800055c8     libredefclass028.obj
 0002:000005d8       ??_C@_0L@LNHEOAOO@unknown_16@ 00000001800055d8     libredefclass028.obj
 0002:000005e8       ??_C@_0L@KEGPNBKP@unknown_17@ 00000001800055e8     libredefclass028.obj
 0002:000005f8       ??_C@_0L@CDPHMNGA@unknown_18@ 00000001800055f8     libredefclass028.obj
 0002:00000608       ??_C@_0L@DKOMPMCB@unknown_19@ 0000000180005608     libredefclass028.obj
 0002:00000618       ??_C@_0L@OJGIPJDB@unknown_20@ 0000000180005618     libredefclass028.obj
 0002:00000628       ??_C@_0CA@KAOFNDEM@JVMTI_HEAP_REFERENCE_JNI_GLOBAL@ 0000000180005628     libredefclass028.obj
 0002:00000648       ??_C@_0CC@HPFAJBK@JVMTI_HEAP_REFERENCE_SYSTEM_CLA@ 0000000180005648     libredefclass028.obj
 0002:00000670       ??_C@_0BN@FDEGFOHC@JVMTI_HEAP_REFERENCE_MONITOR@ 0000000180005670     libredefclass028.obj
 0002:00000690       ??_C@_0CB@HKIBCMAJ@JVMTI_HEAP_REFERENCE_STACK_LOCA@ 0000000180005690     libredefclass028.obj
 0002:000006b8       ??_C@_0BP@EAACMMOE@JVMTI_HEAP_REFERENCE_JNI_LOCAL@ 00000001800056b8     libredefclass028.obj
 0002:000006d8       ??_C@_0BM@IJDEOGOE@JVMTI_HEAP_REFERENCE_THREAD@ 00000001800056d8     libredefclass028.obj
 0002:000006f8       ??_C@_0BL@EDGPPKC@JVMTI_HEAP_REFERENCE_OTHER@ 00000001800056f8     libredefclass028.obj
 0002:00000714       ??_C@_04BCJPDBDA@Code@     0000000180005714     libredefclass028.obj
 0002:00000720       ??_C@_0BA@OCLMCFKC@LineNumberTable@ 0000000180005720     libredefclass028.obj
 0002:00000730       ??_C@_0BD@CPAEPILC@LocalVariableTable@ 0000000180005730     libredefclass028.obj
 0002:00000748       ??_C@_0BH@NMBDNHBD@LocalVariableTypeTable@ 0000000180005748     libredefclass028.obj
 0002:00000760       ??_C@_0O@HIHEEDNJ@StackMapTable@ 0000000180005760     libredefclass028.obj
 0002:00000770       ??_C@_0BH@JHCEFIFG@redefclass028HotMethod@ 0000000180005770     libredefclass028.obj
 0002:00000788       ??_C@_04PFANPMCN@?$CII?$CJV@ 0000000180005788     libredefclass028.obj
 0002:00000790       ??_C@_0L@HCDIAMJG@?9?5?$CFs?0?5?$CFd?3?5@ 0000000180005790     libredefclass028.obj
 0002:000007a0       ??_C@_0JI@HLPECLFI@?$CD?5?4?4?4?6?$CD?5ERROR?3?5too?5many?5complai@ 00000001800057a0     libredefclass028.obj
 0002:00000840       ??_C@_0ED@JNEKCCOB@The?5following?5fake?5exception?5st@ 0000000180005840     libredefclass028.obj
 0002:00000888       ??_C@_0CN@FCNMDFBH@nsk?4share?4Fake_Exception_for_RU@ 0000000180005888     libredefclass028.obj
 0002:000008b8       ??_C@_08PGFFNAEI@?$CI?$CFs?3?$CFd?$CJ?5@ 00000001800058b8     libredefclass028.obj
 0002:000008c8       ??_C@_0DP@IENMAEGI@s?2test?2hotspot?2jtreg?2vmTestbase@ 00000001800058c8     libredefclass028.obj
 0002:00000908       ??_C@_0BL@NDJLFFJB@?7at?5nsk_lvcomplain?$CI?$CFs?3?$CFd?$CJ?6@ 0000000180005908     libredefclass028.obj
 0002:00000928       ??_C@_0BC@JOOKAFKF@?$CD?5ERROR?3?5?$CFs?0?5?$CFd?3?5@ 0000000180005928     libredefclass028.obj
 0002:00000940       ??_C@_09KJEAHMEH@?$CD?5ERROR?3?5@ 0000000180005940     libredefclass028.obj
 0002:0000094c       ??_C@_02GPIOPFAK@?$DO?$DO@ 000000018000594c     libredefclass028.obj
 0002:00000950       ??_C@_02FODMEDOG@?$DM?$DM@ 0000000180005950     libredefclass028.obj
 0002:00000954       ??_C@_02DJGKEECL@?4?4@     0000000180005954     libredefclass028.obj
 0002:00000958       ??_C@_0O@CJPGJOAF@?9?5?$CFs?0?5?$CFd?3?5?$CFs?5@ 0000000180005958     libredefclass028.obj
 0002:00000968       ??_C@_0CB@IAKPDOIC@?$CD?5?5?5verified?5assertion?5is?5FALSE@ 0000000180005968     libredefclass028.obj
 0002:00000990       ??_C@_0CO@LGONDEPD@stdout?3?5fflush?5failed?5?9?5err?$DN?$CFd?5@ 0000000180005990     libredefclass028.obj
 0002:000009c0       ??_C@_0CO@KBGKJPBD@stderr?3?5fflush?5failed?5?9?5err?$DN?$CFd?5@ 00000001800059c0     libredefclass028.obj
 0002:000009f0       ??_C@_0BB@JCNMKLLK@JVMTI_ERROR_NONE@ 00000001800059f0     libredefclass028.obj
 0002:00000a08       ??_C@_0BL@LDIMKLPH@JVMTI_ERROR_INVALID_THREAD@ 0000000180005a08     libredefclass028.obj
 0002:00000a28       ??_C@_0CB@PJFPAIKJ@JVMTI_ERROR_INVALID_THREAD_GROU@ 0000000180005a28     libredefclass028.obj
 0002:00000a50       ??_C@_0BN@LLMKHMNF@JVMTI_ERROR_INVALID_PRIORITY@ 0000000180005a50     libredefclass028.obj
 0002:00000a70       ??_C@_0CB@MBOFKAGB@JVMTI_ERROR_THREAD_NOT_SUSPENDE@ 0000000180005a70     libredefclass028.obj
 0002:00000a98       ??_C@_0BN@FABOLPBI@JVMTI_ERROR_THREAD_SUSPENDED@ 0000000180005a98     libredefclass028.obj
 0002:00000ab8       ??_C@_0BN@FDGNOBJM@JVMTI_ERROR_THREAD_NOT_ALIVE@ 0000000180005ab8     libredefclass028.obj
 0002:00000ad8       ??_C@_0BL@GOBIFKNJ@JVMTI_ERROR_INVALID_OBJECT@ 0000000180005ad8     libredefclass028.obj
 0002:00000af8       ??_C@_0BK@FCMAJPPC@JVMTI_ERROR_INVALID_CLASS@ 0000000180005af8     libredefclass028.obj
 0002:00000b18       ??_C@_0BP@IKLLBKEB@JVMTI_ERROR_CLASS_NOT_PREPARED@ 0000000180005b18     libredefclass028.obj
 0002:00000b38       ??_C@_0BN@KLPPLKG@JVMTI_ERROR_INVALID_METHODID@ 0000000180005b38     libredefclass028.obj
 0002:00000b58       ??_C@_0BN@BCEKOKND@JVMTI_ERROR_INVALID_LOCATION@ 0000000180005b58     libredefclass028.obj
 0002:00000b78       ??_C@_0BM@DFDGPME@JVMTI_ERROR_INVALID_FIELDID@ 0000000180005b78     libredefclass028.obj
 0002:00000b98       ??_C@_0BL@NELIEPEC@JVMTI_ERROR_NO_MORE_FRAMES@ 0000000180005b98     libredefclass028.obj
 0002:00000bb8       ??_C@_0BJ@BDBECFDM@JVMTI_ERROR_OPAQUE_FRAME@ 0000000180005bb8     libredefclass028.obj
 0002:00000bd8       ??_C@_0BK@MIIFNLOB@JVMTI_ERROR_TYPE_MISMATCH@ 0000000180005bd8     libredefclass028.obj
 0002:00000bf8       ??_C@_0BJ@HPCAOILC@JVMTI_ERROR_INVALID_SLOT@ 0000000180005bf8     libredefclass028.obj
 0002:00000c18       ??_C@_0BG@CHILOPNI@JVMTI_ERROR_DUPLICATE@ 0000000180005c18     libredefclass028.obj
 0002:00000c30       ??_C@_0BG@DIEMLHKM@JVMTI_ERROR_NOT_FOUND@ 0000000180005c30     libredefclass028.obj
 0002:00000c48       ??_C@_0BM@NHMCKHOB@JVMTI_ERROR_INVALID_MONITOR@ 0000000180005c48     libredefclass028.obj
 0002:00000c68       ??_C@_0BO@PPEDAJGL@JVMTI_ERROR_NOT_MONITOR_OWNER@ 0000000180005c68     libredefclass028.obj
 0002:00000c88       ??_C@_0BG@FCAIPEID@JVMTI_ERROR_INTERRUPT@ 0000000180005c88     libredefclass028.obj
 0002:00000ca0       ??_C@_0CB@EGDBNKOI@JVMTI_ERROR_INVALID_CLASS_FORMA@ 0000000180005ca0     libredefclass028.obj
 0002:00000cc8       ??_C@_0CG@DGKOGIAL@JVMTI_ERROR_CIRCULAR_CLASS_DEFI@ 0000000180005cc8     libredefclass028.obj
 0002:00000cf0       ??_C@_0BP@ICEALPKC@JVMTI_ERROR_FAILS_VERIFICATION@ 0000000180005cf0     libredefclass028.obj
 0002:00000d10       ??_C@_0DC@JDACLMIO@JVMTI_ERROR_UNSUPPORTED_REDEFIN@ 0000000180005d10     libredefclass028.obj
 0002:00000d48       ??_C@_0DE@GKDKNOMJ@JVMTI_ERROR_UNSUPPORTED_REDEFIN@ 0000000180005d48     libredefclass028.obj
 0002:00000d80       ??_C@_0BO@LAFKIOG@JVMTI_ERROR_INVALID_TYPESTATE@ 0000000180005d80     libredefclass028.obj
 0002:00000da0       ??_C@_0DH@INDGCLLB@JVMTI_ERROR_UNSUPPORTED_REDEFIN@ 0000000180005da0     libredefclass028.obj
 0002:00000dd8       ??_C@_0DE@NHEOMMGI@JVMTI_ERROR_UNSUPPORTED_REDEFIN@ 0000000180005dd8     libredefclass028.obj
 0002:00000e10       ??_C@_0CA@EKPNJOEP@JVMTI_ERROR_UNSUPPORTED_VERSION@ 0000000180005e10     libredefclass028.obj
 0002:00000e30       ??_C@_0BN@OFFMAHHL@JVMTI_ERROR_NAMES_DONT_MATCH@ 0000000180005e30     libredefclass028.obj
 0002:00000e50       ??_C@_0DN@HHBBLAKE@JVMTI_ERROR_UNSUPPORTED_REDEFIN@ 0000000180005e50     libredefclass028.obj
 0002:00000e90       ??_C@_0DO@HMBGBGNA@JVMTI_ERROR_UNSUPPORTED_REDEFIN@ 0000000180005e90     libredefclass028.obj
 0002:00000ed0       ??_C@_0BP@PBECGKHJ@JVMTI_ERROR_UNMODIFIABLE_CLASS@ 0000000180005ed0     libredefclass028.obj
 0002:00000ef0       ??_C@_0BK@CANILEHF@JVMTI_ERROR_NOT_AVAILABLE@ 0000000180005ef0     libredefclass028.obj
 0002:00000f10       ??_C@_0CE@INJKMEFK@JVMTI_ERROR_MUST_POSSESS_CAPABI@ 0000000180005f10     libredefclass028.obj
 0002:00000f38       ??_C@_0BJ@LBFPFPDM@JVMTI_ERROR_NULL_POINTER@ 0000000180005f38     libredefclass028.obj
 0002:00000f58       ??_C@_0BP@CHJPNNEM@JVMTI_ERROR_ABSENT_INFORMATION@ 0000000180005f58     libredefclass028.obj
 0002:00000f78       ??_C@_0BP@OMFMNLC@JVMTI_ERROR_INVALID_EVENT_TYPE@ 0000000180005f78     libredefclass028.obj
 0002:00000f98       ??_C@_0BN@BIBNPHHO@JVMTI_ERROR_ILLEGAL_ARGUMENT@ 0000000180005f98     libredefclass028.obj
 0002:00000fb8       ??_C@_0BK@KKNDHDCE@JVMTI_ERROR_NATIVE_METHOD@ 0000000180005fb8     libredefclass028.obj
 0002:00000fd8       ??_C@_0BK@PMKCFHAE@JVMTI_ERROR_OUT_OF_MEMORY@ 0000000180005fd8     libredefclass028.obj
 0002:00000ff8       ??_C@_0BK@NNJBDMNB@JVMTI_ERROR_ACCESS_DENIED@ 0000000180005ff8     libredefclass028.obj
 0002:00001018       ??_C@_0BI@GHECLMNC@JVMTI_ERROR_WRONG_PHASE@ 0000000180006018     libredefclass028.obj
 0002:00001030       ??_C@_0BF@OLIHJOII@JVMTI_ERROR_INTERNAL@ 0000000180006030     libredefclass028.obj
 0002:00001048       ??_C@_0BO@EOHGKJHI@JVMTI_ERROR_UNATTACHED_THREAD@ 0000000180006048     libredefclass028.obj
 0002:00001068       ??_C@_0CA@LKHFDACL@JVMTI_ERROR_INVALID_ENVIRONMENT@ 0000000180006068     libredefclass028.obj
 0002:00001088       ??_C@_0BA@MMFHLOKK@?$DMunknown?5error?$DO@ 0000000180006088     libredefclass028.obj
 0002:00001098       ??_C@_0CF@CBHOKDB@throwable?5?$DN?5jni?9?$DOExceptionOccur@ 0000000180006098     libredefclass028.obj
 0002:000010c0       ??_C@_03OFAPEBGM@?$CFs?6@  00000001800060c0     libredefclass028.obj
 0002:000010c8       ??_C@_0DM@LPIGEGNJ@s?2test?2hotspot?2jtreg?2vmTestbase@ 00000001800060c8     libredefclass028.obj
 0002:00001108       ??_C@_0CC@NFCNPEPK@Exception?5in?5JNI?5call?5?$CIcleared?$CJ@ 0000000180006108     libredefclass028.obj
 0002:00001130       ??_C@_0BJ@IBAKFIKF@jni?9?$DOExceptionDescribe?$CI?$CJ@ 0000000180006130     libredefclass028.obj
 0002:00001150       ??_C@_0BG@GGKALKMH@jni?9?$DOExceptionClear?$CI?$CJ@ 0000000180006150     libredefclass028.obj
 0002:00001168       ??_C@_0CF@JMGFGJLJ@?$CD?5?5?5verified?5JNI?5assertion?5is?5F@ 0000000180006168     libredefclass028.obj
 0002:00001190       ??_C@_07KBAMPNJK@verbose@  0000000180006190     libredefclass028.obj
 0002:00001198       ??_C@_0DN@PKJBOLAP@nsk_jvmti_parseOptions?$CI?$CJ?3?5unexp@ 0000000180006198     libredefclass028.obj
 0002:000011d8       ??_C@_05IMBNNINJ@trace@    00000001800061d8     libredefclass028.obj
 0002:000011e0       ??_C@_0DD@BJKGNDMB@nsk_jvmti_parseOptions?$CI?$CJ?3?5no?5va@ 00000001800061e0     libredefclass028.obj
 0002:00001214       ??_C@_04CGFJFPFD@none@     0000000180006214     libredefclass028.obj
 0002:0000121c       ??_C@_06BMELKFMA@before@   000000018000621c     libredefclass028.obj
 0002:00001224       ??_C@_05CMKPCFDK@after@    0000000180006224     libredefclass028.obj
 0002:0000122c       ??_C@_03NFKEKGGK@all@      000000018000622c     libredefclass028.obj
 0002:00001230       ??_C@_0DM@NDNJGJKE@nsk_jvmti_parseOptions?$CI?$CJ?3?5uexpe@ 0000000180006230     libredefclass028.obj
 0002:00001270       ??_C@_08NBBJKJO@waittime@  0000000180006270     libredefclass028.obj
 0002:00001280       ??_C@_0DO@CMHGAOHC@nsk_jvmti_parseOptions?$CI?$CJ?3?5not?5i@ 0000000180006280     libredefclass028.obj
 0002:000012c0       ??_C@_0DL@LNMPBDLN@nsk_jvmti_parseOptions?$CI?$CJ?3?5negat@ 00000001800062c0     libredefclass028.obj
 0002:00001300       ??_C@_0DA@GMFJNOJH@nsk_jvmti_parseOptions?$CI?$CJ?3?5unkno@ 0000000180006300     libredefclass028.obj
 0002:00001330       ??_C@_0CO@CCIAMEAN@nsk_jvmti_parseOptions?$CI?$CJ?3?5found@ 0000000180006330     libredefclass028.obj
 0002:00001360       ??_C@_0CJ@OEGPCGDL@nsk_jvmti_parseOptions?$CI?$CJ?3?5out?5o@ 0000000180006360     libredefclass028.obj
 0002:00001390       ??_C@_0DI@NMBHPGGF@nsk_jvmti_parseOptions?$CI?$CJ?3?5too?5m@ 0000000180006390     libredefclass028.obj
 0002:000013c8       ??_C@_03POGCGECB@?5?0?$HO@ 00000001800063c8     libredefclass028.obj
 0002:000013d0       ??_C@_0CB@MLNJNCLJ@?5?5jvmti?5error?3?5code?$DN?$CFd?0?5name?$DN?$CFs@ 00000001800063d0     libredefclass028.obj
 0002:000013f8       ??_C@_0CD@OHBGDKMK@?$CD?5?5?5jvmti?5error?3?5code?$DN?$CFd?0?5name?$DN@ 00000001800063f8     libredefclass028.obj
 0002:00001420       ??_C@_0CG@JNNCGPHB@?$CD?5?5?5error?5expected?3?5code?$DN?$CFd?0?5na@ 0000000180006420     libredefclass028.obj
 0002:00001450       ??_C@_0EB@IMGKPCGE@?$CIstr_obj?5?$DN?5jni?9?$DONewStringUTF?$CIco@ 0000000180006450     libredefclass028.obj
 0002:000014a0       ??_C@_0EA@HFOGGBCC@s?2test?2hotspot?2jtreg?2vmTestbase@ 00000001800064a0     libredefclass028.obj
 0002:000014e0       ??_C@_05KKCIMGE@error@     00000001800064e0     libredefclass028.obj
 0002:000014e8       ??_C@_0CJ@JACLEAA@Test?5failed?5by?5setFailStatus?$CI?$CJ?4@ 00000001800064e8     libredefclass028.obj
 0002:00001518       ??_C@_0BD@HGNAOMCP@agent_data_monitor@ 0000000180006518     libredefclass028.obj
 0002:00001530       ??_C@_0EB@OGCLGKLN@javaVM?9?$DOGetEnv?$CI?$CIvoid?5?$CK?$CK?$CJ?$CGjvmti_@ 0000000180006530     libredefclass028.obj
 0002:00001580       ??_C@_0EA@PNBCDMOA@s?2test?2hotspot?2jtreg?2vmTestbase@ 0000000180006580     libredefclass028.obj
 0002:000015c0       ??_C@_0CI@DDPIFBGM@init_agent_data?$CIjvmti_env?0?5?$CGage@ 00000001800065c0     libredefclass028.obj
 0002:000015e8       ??_C@_0DI@ILAHDLMP@?$CI?$CKagentThreadProc?$CJ?$CIjvmti_env?0?5a@ 00000001800065e8     libredefclass028.obj
 0002:00001620       ??_C@_0BD@KDBALNLB@JVMTI?5agent?5thread@ 0000000180006620     libredefclass028.obj
 0002:00001638       ??_C@_0BB@NOKBFPFO@java?1lang?1Thread@ 0000000180006638     libredefclass028.obj
 0002:0000164c       ??_C@_06FALKBLGB@?$DMinit?$DO@ 000000018000664c     libredefclass028.obj
 0002:00001658       ??_C@_0BG@IKDDPPGD@?$CILjava?1lang?1String?$DL?$CJV@ 0000000180006658     libredefclass028.obj
 0002:00001670       ??_C@_0EB@IFJBFEKC@?$CIthreadClass?5?$DN?5jni_env?9?$DOFindCla@ 0000000180006670     libredefclass028.obj
 0002:000016c0       ??_C@_0GF@FGFIBKKL@?$CIthreadCtor?5?$DN?5jni_env?9?$DOGetMetho@ 00000001800066c0     libredefclass028.obj
 0002:00001728       ??_C@_0DN@NCPDJLOG@?$CIthreadName?5?$DN?5jni_env?9?$DONewStrin@ 0000000180006728     libredefclass028.obj
 0002:00001770       ??_C@_0FE@PFKODBGC@?$CIthreadObject?5?$DN?5jni_env?9?$DONewObj@ 0000000180006770     libredefclass028.obj
 0002:000017d0       ??_C@_0ED@HOBAHHJI@?$CIthreadGlobalRef?5?$DN?5jni_env?9?$DONew@ 00000001800067d0     libredefclass028.obj
 0002:00001820       ??_C@_0FN@HNJJAHFC@jvmti_env?9?$DORunAgentThread?$CIagent@ 0000000180006820     libredefclass028.obj
 0002:00001880       ??_C@_0EA@MOJDNKDF@Debuggee?5status?5sync?5aborted?5be@ 0000000180006880     libredefclass028.obj
 0002:000018c0       ??_C@_0CO@PGPGMHBJ@No?5status?5sync?5occured?5for?5time@ 00000001800068c0     libredefclass028.obj
 0002:000018f0       ??_C@_0CL@DOEBDPKJ@Debuggee?5was?5not?5suspended?5on?5s@ 00000001800068f0     libredefclass028.obj
 0002:00001920       ??_C@_0EA@EEOEJAEN@status?5?$DN?5syncDebuggeeStatus?$CIjni@ 0000000180006920     libredefclass028.obj
 0002:00001960       ??_C@_0BL@JBCFNBMB@nsk_jvmti_resetAgentData?$CI?$CJ@ 0000000180006960     libredefclass028.obj
 0002:00001980       ??_C@_0DN@NNGECJON@jvmti_env?9?$DOSetEventNotification@ 0000000180006980     libredefclass028.obj
 0002:000019c0       ??_C@_0EL@LPBEELIP@s?2test?2hotspot?2jtreg?2vmTestbase@ 00000001800069c0     libredefclass028.obj
 0002:00001a10       ??_C@_0CK@JDAMFDMJ@jvmti?9?$DOSetTag?$CIo?0?5tag?$CJ?5?$DN?$DN?5JVMTI_@ 0000000180006a10     libredefclass028.obj
 0002:00001a40       ??_C@_0CC@DAMNHKNI@Can?8t?5set?5tag?5?$CFli?5for?5object?5?$CFl@ 0000000180006a40     libredefclass028.obj
 0002:00001a68       ??_C@_0DL@HAJPNKEF@jvmti?9?$DOGetObjectHashCode?$CIo?0?5?$CGha@ 0000000180006a68     libredefclass028.obj
 0002:00001aa8       ??_C@_0BL@JFPIEOBF@Can?8t?5get?5hash?5object?5?$CFlx?6@ 0000000180006aa8     libredefclass028.obj
 0002:00001ac8       ??_C@_0BG@DICPHBKN@setTag?3?5?$CF08x?5?$DM?9?5?$CF?53li@ 0000000180006ac8     libredefclass028.obj
 0002:00001ae0       ??_C@_0DH@FCEEBDMJ@?$CIs?5?$DN?5jni?9?$DOGetStringUTFChars?$CIsIn@ 0000000180006ae0     libredefclass028.obj
 0002:00001b18       ??_C@_0BJ@OKKGHDCN@Can?8t?5get?5string?5at?5?$CF?$CDp?6@ 0000000180006b18     libredefclass028.obj
 0002:00001b38       ??_C@_0BP@EKFLGGFJ@Can?8t?5get?5string?5at?5?$CF?$CDp?3?5null?6@ 0000000180006b38     libredefclass028.obj
 0002:00001b58       ??_C@_06ICODBHCL@?5?1?1?5?$CFs@ 0000000180006b58     libredefclass028.obj
 0002:00001b60       ??_C@_0DB@KGFPLEGO@?$CIr?5?$DN?5jvmti?9?$DOGetTag?$CIo?0?5?$CGtag?$CJ?$CJ?5?$DN?$DN@ 0000000180006b60     libredefclass028.obj
 0002:00001b98       ??_C@_0CO@PDAGBCGJ@Can?8t?5GetTag?5for?5object?5?$CFlx?4?5Re@ 0000000180006b98     libredefclass028.obj
 0002:00001bc8       ??_C@_0CH@HPEODOHC@TEST_BUG?3?5Max?4?5number?5of?5refs?5r@ 0000000180006bc8     libredefclass028.obj
 0002:00001bf0       ??_C@_0DI@PHFCABIM@?$CIr?5?$DN?5jvmti?9?$DOGetTag?$CIfrom?0?5?$CGtagFr@ 0000000180006bf0     libredefclass028.obj
 0002:00001c28       ??_C@_0DI@MDEGFNKD@TEST_BUG?3?5Can?8t?5GetTag?5for?5obje@ 0000000180006c28     libredefclass028.obj
 0002:00001c60       ??_C@_0DE@MLELJAHM@?$CIr?5?$DN?5jvmti?9?$DOGetTag?$CIto?0?5?$CGtagTo?$CJ?$CJ@ 0000000180006c60     libredefclass028.obj
 0002:00001c98       ??_C@_0CK@EOPGBGKK@isRedefinitionOccurred?5is?5calle@ 0000000180006c98     libredefclass028.obj
 0002:00001cd0       ??_C@_0FK@GLBEEMAL@s?2test?2hotspot?2jtreg?2vmTestbase@ 0000000180006cd0     libredefclass028.obj
 0002:00001d30       ??_C@_0BN@NEEOIPLO@notifyNativeAgent?5is?5called?6@ 0000000180006d30     libredefclass028.obj
 0002:00001d50       ??_C@_0CI@GOIGCOJA@CompiledMethodLoad?5event?5receiv@ 0000000180006d50     libredefclass028.obj
 0002:00001d78       ??_C@_0DH@GCOJDBIO@jvmti_env?9?$DOGetMethodName?$CImethod@ 0000000180006d78     libredefclass028.obj
 0002:00001db0       ??_C@_0ID@FKGELPPN@?7method?3?5name?$DN?$CC?$CFs?$CC?5signature?$DN?$CC?$CF@ 0000000180006db0     libredefclass028.obj
 0002:00001e38       ??_C@_0DD@CIFOBJCN@CompiledMethodLoad?3?5a?5tested?5ho@ 0000000180006e38     libredefclass028.obj
 0002:00001e70       ??_C@_0DI@DJLHKDHD@Compilation?5occured?5before?5meth@ 0000000180006e70     libredefclass028.obj
 0002:00001ea8       ??_C@_0CF@NAKKFALD@CompiledMethodUnload?5event?5rece@ 0000000180006ea8     libredefclass028.obj
 0002:00001ed0       ??_C@_0DN@NNJMMNHN@for?3?5?7method?3?5name?$DN?$CC?$CFs?$CC?5signatu@ 0000000180006ed0     libredefclass028.obj
 0002:00001f10       ??_C@_0DM@NNJEKMJH@agentProc?3?5waiting?5for?5the?5debu@ 0000000180006f10     libredefclass028.obj
 0002:00001f50       ??_C@_0CH@NCEJGEND@agentProc?3?5resuming?5the?5debugge@ 0000000180006f50     libredefclass028.obj
 0002:00001f80       ??_C@_0EB@BIIGAOGH@agentProc?3?5sending?5all?5generate@ 0000000180006f80     libredefclass028.obj
 0002:00001fc8       ??_C@_0DI@BFMHPNME@jvmti?9?$DOGenerateEvents?$CIJVMTI_EVE@ 0000000180006fc8     libredefclass028.obj
 0002:00002000       ??_C@_0DH@DPOOGNHJ@agentProc?3?5waiting?5for?5hotspot?5@ 0000000180007000     libredefclass028.obj
 0002:00002040       ??_C@_0GO@BBNMOEDN@WARNING?3?5CompiledMethodLoad?5eve@ 0000000180007040     libredefclass028.obj
 0002:000020b0       ??_C@_0CF@BBGBFFAI@agentProc?3?5hotspot?5method?5compi@ 00000001800070b0     libredefclass028.obj
 0002:000020d8       ??_C@_0DK@PKJDKBKO@jvmti_env?9?$DOGetMethodDeclaringCl@ 00000001800070d8     libredefclass028.obj
 0002:00002118       ??_C@_0DK@LDGEOOHJ@jvmti_env?9?$DOGetClassSignature?$CIde@ 0000000180007118     libredefclass028.obj
 0002:00002158       ??_C@_0DC@NHCDKGHH@agentProc?3?5hotspot?5method?5class@ 0000000180007158     libredefclass028.obj
 0002:00002190       ??_C@_0EI@KJBONIIM@agentProc?3?5?$DO?$DO?$DO?$DO?$DO?$DO?$DO?$DO?5Invoke?5Rede@ 0000000180007190     libredefclass028.obj
 0002:000021d8       ??_C@_0CF@OBOBAJEI@jvmti?9?$DORedefineClasses?$CI1?0?5?$CGclas@ 00000001800071d8     libredefclass028.obj
 0002:00002200       ??_C@_0DM@OBAGCLFD@agentProc?3?5?$DM?$DM?$DM?$DM?$DM?$DM?$DM?$DM?5RedefineCla@ 0000000180007200     libredefclass028.obj
 0002:00002240       ??_C@_0DN@KDPOPOJI@agentProc?3?5waiting?5for?5the?5debu@ 0000000180007240     libredefclass028.obj
 0002:00002280       ??_C@_0DA@MJHFJKIM@agentProc?3?5final?5resuming?5of?5th@ 0000000180007280     libredefclass028.obj
 0002:000022b0       ??_C@_0BG@FMNKMBB@agentProc?3?5finished?6?6@ 00000001800072b0     libredefclass028.obj
 0002:000022c8       ??_C@_0CA@MNKGCBCG@nsk_jvmti_parseOptions?$CIoptions?$CJ@ 00000001800072c8     libredefclass028.obj
 0002:000022e8       ??_C@_0BD@FAKCJAOH@waittime?$DN?$CFd?5msecs?6@ 00000001800072e8     libredefclass028.obj
 0002:00002300       ??_C@_0DN@MIAMNFPH@?$CIjvmti?5?$DN?5nsk_jvmti_createJVMTIE@ 0000000180007300     libredefclass028.obj
 0002:00002340       ??_C@_0BO@DBKDIPGD@jvmti?9?$DOAddCapabilities?$CI?$CGcaps?$CJ@ 0000000180007340     libredefclass028.obj
 0002:00002360       ??_C@_0BN@HGIKGGD@setting?5event?5callbacks?5?4?4?4?6@ 0000000180007360     libredefclass028.obj
 0002:00002380       ??_C@_0DI@NJCFGEGC@jvmti?9?$DOSetEventCallbacks?$CI?$CGcallb@ 0000000180007380     libredefclass028.obj
 0002:000023b8       ??_C@_0DC@EEJJNFPC@setting?5event?5callbacks?5done?6en@ 00000001800073b8     libredefclass028.obj
 0002:000023f0       ??_C@_0BL@GBOGNFCP@enabling?5the?5events?5done?6?6@ 00000001800073f0     libredefclass028.obj
 0002:00002410       ??_C@_0CL@PIACJIPK@nsk_jvmti_setAgentProc?$CIagentPro@ 0000000180007410     libredefclass028.obj
 0002:00002450       ??_C@_1EC@JIJBPKFM@?$AAa?$AAp?$AAi?$AA?9?$AAm?$AAs?$AA?9?$AAw?$AAi?$AAn?$AA?9?$AAc?$AAo?$AAr?$AAe@ 0000000180007450     MSVCRT:thread_safe_statics.obj
 0002:00002498       ??_C@_1BK@MGMFAEKH@?$AAk?$AAe?$AAr?$AAn?$AAe?$AAl?$AA3?$AA2?$AA?4?$AAd?$AAl?$AAl@ 0000000180007498     MSVCRT:thread_safe_statics.obj
 0002:000024b8       ??_C@_0BJ@JEBJOJFJ@SleepConditionVariableCS@ 00000001800074b8     MSVCRT:thread_safe_statics.obj
 0002:000024d8       ??_C@_0BJ@PGPPEPCC@WakeAllConditionVariable@ 00000001800074d8     MSVCRT:thread_safe_statics.obj
 0002:000024f8       _pDefaultRawDllMain        00000001800074f8     MSVCRT:dll_dllmain.obj
 0002:000024f8       _pRawDllMain               00000001800074f8     MSVCRT:dll_dllmain.obj
 0002:00002500       __xmm@ffffffffffffffffffffffffffffffff 0000000180007500     MSVCRT:utility.obj
 0002:00002510       _load_config_used          0000000180007510     MSVCRT:loadcfg.obj
 0002:00002700       _tls_used                  0000000180007700     MSVCRT:tlssup.obj
 0002:00002728       __volatile_metadata        0000000180007728     <linker-defined>
 0002:00002b18       __rtc_iaa                  0000000180007b18     MSVCRT:initsect.obj
 0002:00002b20       __rtc_izz                  0000000180007b20     MSVCRT:initsect.obj
 0002:00002b28       __rtc_taa                  0000000180007b28     MSVCRT:initsect.obj
 0002:00002b30       __rtc_tzz                  0000000180007b30     MSVCRT:initsect.obj
 0002:00002b38       _tls_start                 0000000180007b38     MSVCRT:tlssup.obj
 0002:00002b3c       _Init_thread_epoch         0000000180007b3c     MSVCRT:thread_safe_statics.obj
 0002:00002b40       _tls_end                   0000000180007b40     MSVCRT:tlssup.obj
 0002:00003334       __IMPORT_DESCRIPTOR_KERNEL32 0000000180008334     kernel32:KERNEL32.dll
 0002:00003348       __IMPORT_DESCRIPTOR_VCRUNTIME140 0000000180008348     vcruntime:VCRUNTIME140.dll
 0002:0000335c       __IMPORT_DESCRIPTOR_api-ms-win-crt-heap-l1-1-0 000000018000835c     ucrt:api-ms-win-crt-heap-l1-1-0.dll
 0002:00003370       __IMPORT_DESCRIPTOR_api-ms-win-crt-runtime-l1-1-0 0000000180008370     ucrt:api-ms-win-crt-runtime-l1-1-0.dll
 0002:00003384       __IMPORT_DESCRIPTOR_api-ms-win-crt-convert-l1-1-0 0000000180008384     ucrt:api-ms-win-crt-convert-l1-1-0.dll
 0002:00003398       __IMPORT_DESCRIPTOR_api-ms-win-crt-stdio-l1-1-0 0000000180008398     ucrt:api-ms-win-crt-stdio-l1-1-0.dll
 0002:000033ac       __IMPORT_DESCRIPTOR_api-ms-win-crt-string-l1-1-0 00000001800083ac     ucrt:api-ms-win-crt-string-l1-1-0.dll
 0002:000033c0       __NULL_IMPORT_DESCRIPTOR   00000001800083c0     kernel32:KERNEL32.dll
 0003:00000048       _Init_global_epoch         0000000180009048     MSVCRT:thread_safe_statics.obj
 0003:00000050       __security_cookie          0000000180009050     MSVCRT:gs_cookie.obj
 0003:00000058       __security_cookie_complement 0000000180009058     MSVCRT:gs_cookie.obj
 0003:00000060       __scrt_native_dllmain_reason 0000000180009060     MSVCRT:utility.obj
 0003:00000068       __isa_available            0000000180009068     MSVCRT:cpu_disp.obj
 0003:0000006c       __isa_enabled              000000018000906c     MSVCRT:cpu_disp.obj
 0003:00000070       __memset_fast_string_threshold 0000000180009070     MSVCRT:cpu_disp.obj
 0003:00000078       __memset_nt_threshold      0000000180009078     MSVCRT:cpu_disp.obj
 0003:00000080       __scrt_ucrt_dll_is_in_use  0000000180009080     MSVCRT:ucrt_stubs.obj
 0003:00000090       g_wrongHeapCallbacks       0000000180009090     libredefclass028.obj
 0003:00000110       g_szTagInfo                0000000180009110     libredefclass028.obj
 0003:00002050       g_tagFlags                 000000018000b050     libredefclass028.obj
 0003:00002438       g_refsToVerifyCnt          000000018000b438     libredefclass028.obj
 0003:0000243c       g_fakeUserData             000000018000b43c     libredefclass028.obj
 0003:00002440       g_tagVisitCount            000000018000b440     libredefclass028.obj
 0003:000033e0       g_refsToVerify             000000018000c3e0     libredefclass028.obj
 0003:0001aae0       g_userDataError            0000000180023ae0     libredefclass028.obj
 0003:0001aca0       ?_OptionsStorage@?1??__local_stdio_printf_options@@9@4_KA 0000000180023ca0     libredefclass028.obj
 0003:0001b268       _tls_index                 0000000180024268     MSVCRT:tlssup.obj
 0003:0001b270       __scrt_current_native_startup_state 0000000180024270     MSVCRT:utility.obj
 0003:0001b278       __scrt_native_startup_lock 0000000180024278     MSVCRT:utility.obj
 0003:0001b2b8       __scrt_debugger_hook_flag  00000001800242b8     MSVCRT:utility_desktop.obj
 0003:0001b2c0       ?__type_info_root_node@@3U__type_info_node@@A 00000001800242c0     MSVCRT:tncleanup.obj
 0003:0001b2d0       ?_OptionsStorage@?1??__local_stdio_scanf_options@@9@4_KA 00000001800242d0     MSVCRT:default_local_stdio_options.obj
 0003:0001b2d8       __favor                    00000001800242d8     MSVCRT:cpu_disp.obj
 0003:0001b2e0       __dyn_tls_init_callback    00000001800242e0     <common>

 entry point at        0001:000031a0

 Static symbols

 0000:fffd9000       .debug$S                   0000000180000000     redefclass028.exp
 0000:fffd9000       .debug$S                   0000000180000000     vcruntime:VCRUNTIME140.dll
 0000:fffd9000       .debug$S                   0000000180000000     vcruntime:VCRUNTIME140.dll
 0000:fffd9000       .debug$S                   0000000180000000     vcruntime:VCRUNTIME140.dll
 0000:fffd9000       .debug$S                   0000000180000000     vcruntime:VCRUNTIME140.dll
 0000:fffd9000       .debug$S                   0000000180000000     vcruntime:VCRUNTIME140.dll
 0000:fffd9000       .debug$S                   0000000180000000     vcruntime:VCRUNTIME140.dll
 0000:fffd9000       .debug$S                   0000000180000000     vcruntime:VCRUNTIME140.dll
 0000:fffd9000       .debug$S                   0000000180000000     ucrt:api-ms-win-crt-convert-l1-1-0.dll
 0000:fffd9000       .debug$S                   0000000180000000     ucrt:api-ms-win-crt-heap-l1-1-0.dll
 0000:fffd9000       .debug$S                   0000000180000000     ucrt:api-ms-win-crt-heap-l1-1-0.dll
 0000:fffd9000       .debug$S                   0000000180000000     ucrt:api-ms-win-crt-heap-l1-1-0.dll
 0000:fffd9000       .debug$S                   0000000180000000     ucrt:api-ms-win-crt-heap-l1-1-0.dll
 0000:fffd9000       .debug$S                   0000000180000000     ucrt:api-ms-win-crt-runtime-l1-1-0.dll
 0000:fffd9000       .debug$S                   0000000180000000     ucrt:api-ms-win-crt-runtime-l1-1-0.dll
 0000:fffd9000       .debug$S                   0000000180000000     ucrt:api-ms-win-crt-runtime-l1-1-0.dll
 0000:fffd9000       .debug$S                   0000000180000000     ucrt:api-ms-win-crt-runtime-l1-1-0.dll
 0000:fffd9000       .debug$S                   0000000180000000     ucrt:api-ms-win-crt-runtime-l1-1-0.dll
 0000:fffd9000       .debug$S                   0000000180000000     ucrt:api-ms-win-crt-runtime-l1-1-0.dll
 0000:fffd9000       .debug$S                   0000000180000000     ucrt:api-ms-win-crt-runtime-l1-1-0.dll
 0000:fffd9000       .debug$S                   0000000180000000     ucrt:api-ms-win-crt-runtime-l1-1-0.dll
 0000:fffd9000       .debug$S                   0000000180000000     ucrt:api-ms-win-crt-runtime-l1-1-0.dll
 0000:fffd9000       .debug$S                   0000000180000000     ucrt:api-ms-win-crt-runtime-l1-1-0.dll
 0000:fffd9000       .debug$S                   0000000180000000     ucrt:api-ms-win-crt-runtime-l1-1-0.dll
 0000:fffd9000       .debug$S                   0000000180000000     ucrt:api-ms-win-crt-runtime-l1-1-0.dll
 0000:fffd9000       .debug$S                   0000000180000000     ucrt:api-ms-win-crt-runtime-l1-1-0.dll
 0000:fffd9000       .debug$S                   0000000180000000     ucrt:api-ms-win-crt-runtime-l1-1-0.dll
 0000:fffd9000       .debug$S                   0000000180000000     ucrt:api-ms-win-crt-runtime-l1-1-0.dll
 0000:fffd9000       .debug$S                   0000000180000000     ucrt:api-ms-win-crt-runtime-l1-1-0.dll
 0000:fffd9000       .debug$S                   0000000180000000     ucrt:api-ms-win-crt-stdio-l1-1-0.dll
 0000:fffd9000       .debug$S                   0000000180000000     ucrt:api-ms-win-crt-stdio-l1-1-0.dll
 0000:fffd9000       .debug$S                   0000000180000000     ucrt:api-ms-win-crt-stdio-l1-1-0.dll
 0000:fffd9000       .debug$S                   0000000180000000     ucrt:api-ms-win-crt-stdio-l1-1-0.dll
 0000:fffd9000       .debug$S                   0000000180000000     ucrt:api-ms-win-crt-stdio-l1-1-0.dll
 0000:fffd9000       .debug$S                   0000000180000000     ucrt:api-ms-win-crt-stdio-l1-1-0.dll
 0000:fffd9000       .debug$S                   0000000180000000     ucrt:api-ms-win-crt-stdio-l1-1-0.dll
 0000:fffd9000       .debug$S                   0000000180000000     ucrt:api-ms-win-crt-stdio-l1-1-0.dll
 0000:fffd9000       .debug$S                   0000000180000000     ucrt:api-ms-win-crt-stdio-l1-1-0.dll
 0000:fffd9000       .debug$S                   0000000180000000     ucrt:api-ms-win-crt-stdio-l1-1-0.dll
 0000:fffd9000       .debug$S                   0000000180000000     ucrt:api-ms-win-crt-string-l1-1-0.dll
 0000:fffd9000       .debug$S                   0000000180000000     ucrt:api-ms-win-crt-string-l1-1-0.dll
 0000:fffd9000       .debug$S                   0000000180000000     ucrt:api-ms-win-crt-string-l1-1-0.dll
 0000:fffd9000       .debug$S                   0000000180000000     ucrt:api-ms-win-crt-string-l1-1-0.dll
 0000:fffd9000       .debug$S                   0000000180000000     ucrt:api-ms-win-crt-string-l1-1-0.dll
 0000:fffd9000       .debug$S                   0000000180000000     ucrt:api-ms-win-crt-string-l1-1-0.dll
 0000:fffd9000       .debug$S                   0000000180000000     ucrt:api-ms-win-crt-string-l1-1-0.dll
 0000:fffd9000       .debug$S                   0000000180000000     ucrt:api-ms-win-crt-string-l1-1-0.dll
 0000:fffd9000       .debug$S                   0000000180000000     kernel32:KERNEL32.dll
 0000:fffd9000       .debug$S                   0000000180000000     kernel32:KERNEL32.dll
 0000:fffd9000       .debug$S                   0000000180000000     kernel32:KERNEL32.dll
 0000:fffd9000       .debug$S                   0000000180000000     kernel32:KERNEL32.dll
 0000:fffd9000       .debug$S                   0000000180000000     kernel32:KERNEL32.dll
 0000:fffd9000       .debug$S                   0000000180000000     kernel32:KERNEL32.dll
 0000:fffd9000       .debug$S                   0000000180000000     kernel32:KERNEL32.dll
 0000:fffd9000       .debug$S                   0000000180000000     kernel32:KERNEL32.dll
 0000:fffd9000       .debug$S                   0000000180000000     kernel32:KERNEL32.dll
 0000:fffd9000       .debug$S                   0000000180000000     kernel32:KERNEL32.dll
 0000:fffd9000       .debug$S                   0000000180000000     kernel32:KERNEL32.dll
 0000:fffd9000       .debug$S                   0000000180000000     kernel32:KERNEL32.dll
 0000:fffd9000       .debug$S                   0000000180000000     kernel32:KERNEL32.dll
 0000:fffd9000       .debug$S                   0000000180000000     kernel32:KERNEL32.dll
 0000:fffd9000       .debug$S                   0000000180000000     kernel32:KERNEL32.dll
 0000:fffd9000       .debug$S                   0000000180000000     kernel32:KERNEL32.dll
 0000:fffd9000       .debug$S                   0000000180000000     kernel32:KERNEL32.dll
 0000:fffd9000       .debug$S                   0000000180000000     kernel32:KERNEL32.dll
 0000:fffd9000       .debug$S                   0000000180000000     kernel32:KERNEL32.dll
 0000:fffd9000       .debug$S                   0000000180000000     kernel32:KERNEL32.dll
 0000:fffd9000       .debug$S                   0000000180000000     kernel32:KERNEL32.dll
 0000:fffd9000       .debug$S                   0000000180000000     kernel32:KERNEL32.dll
 0000:fffd9000       .debug$S                   0000000180000000     kernel32:KERNEL32.dll
 0000:fffd9000       .debug$S                   0000000180000000     kernel32:KERNEL32.dll
 0000:fffd9000       .debug$S                   0000000180000000     kernel32:KERNEL32.dll
 0000:fffd9000       .debug$S                   0000000180000000     kernel32:KERNEL32.dll
 0000:fffd9000       .debug$S                   0000000180000000     kernel32:KERNEL32.dll
 0000:fffd9000       .debug$S                   0000000180000000     kernel32:KERNEL32.dll
 0001:00001260       addRefToVerify             0000000180002260 f   libredefclass028.obj
 0001:000012cc       agentProc                  00000001800022cc f   libredefclass028.obj
 0001:00001630       agentThreadWrapper         0000000180002630 f   libredefclass028.obj
 0001:0000179c       check_option               000000018000279c f   libredefclass028.obj
 0001:000019e4       file_basename              00000001800029e4 f   libredefclass028.obj
 0001:0000267c       startAgentThreadWrapper    000000018000367c f   libredefclass028.obj
 0001:000029bc       syncDebuggeeStatus         00000001800039bc f   libredefclass028.obj
 0001:00002c5c       capture_previous_context   0000000180003c5c f   MSVCRT:gs_report.obj
 0001:00002cd0       ?__scrt_initialize_thread_safe_statics@@YAHXZ 0000000180003cd0 f   MSVCRT:thread_safe_statics.obj
 0001:00002da0       ?__scrt_uninitialize_thread_safe_statics@@YAXXZ 0000000180003da0 f   MSVCRT:thread_safe_statics.obj
 0001:00002e50       $$000000                   0000000180003e50     MSVCRT:amdsecgs.obj
 0001:00002e80       ?dllmain_crt_dispatch@@YAHQEAUHINSTANCE__@@KQEAX@Z 0000000180003e80 f   MSVCRT:dll_dllmain.obj
 0001:00002ed0       ?dllmain_crt_process_attach@@YAHQEAUHINSTANCE__@@QEAX@Z 0000000180003ed0 f   MSVCRT:dll_dllmain.obj
 0001:00002fe8       ?dllmain_crt_process_detach@@YAH_N@Z 0000000180003fe8 f   MSVCRT:dll_dllmain.obj
 0001:0000306c       ?dllmain_dispatch@@YAHQEAUHINSTANCE__@@KQEAX@Z 000000018000406c f   MSVCRT:dll_dllmain.obj
 0001:00003a80       $$000000                   0000000180004a80     MSVCRT:guard_dispatch.obj
 0001:00003aa0       $$000000                   0000000180004aa0     MSVCRT:guard_xfg_dispatch.obj
 0001:00003ab6       ?fin$0@?0??dllmain_crt_process_attach@@YAHQEAUHINSTANCE__@@QEAX@Z@4HA 0000000180004ab6 f   MSVCRT:dll_dllmain.obj
 0001:00003acd       ?fin$0@?0??dllmain_crt_process_detach@@YAH_N@Z@4HA 0000000180004acd f   MSVCRT:dll_dllmain.obj
 0001:00003ae6       ?fin$1@?0??dllmain_crt_process_detach@@YAH_N@Z@4HA 0000000180004ae6 f   MSVCRT:dll_dllmain.obj
 0001:00003afa       ?filt$0@?0??dllmain_dispatch@@YAHQEAUHINSTANCE__@@KQEAX@Z@4HA 0000000180004afa f   MSVCRT:dll_dllmain.obj
 0001:00003b30       __scrt_is_nonwritable_in_current_image$filt$0 0000000180004b30 f   MSVCRT:utility.obj
 0002:00000220       ?__scrt_initialize_tss_var@@3P6AHXZEA 0000000180005220     MSVCRT:thread_safe_statics.obj
 0002:00000340       ?opcLengths@@3QBEB         0000000180005340     libredefclass028.obj
 0002:00002440       GS_ExceptionPointers       0000000180007440     MSVCRT:gs_report.obj
 0002:00002b48       $unwind$fprintf            0000000180007b48     libredefclass028.obj
 0002:00002b54       $unwind$printf             0000000180007b54     libredefclass028.obj
 0002:00002b60       $unwind$?NewObject@JNIEnv_@@QEAAPEAV_jobject@@PEAV_jclass@@PEAU_jmethodID@@ZZ 0000000180007b60     libredefclass028.obj
 0002:00002b60       $unwind$nsk_lcomplain      0000000180007b60     libredefclass028.obj
 0002:00002b60       $unwind$nsk_ldisplay       0000000180007b60     libredefclass028.obj
 0002:00002b68       $unwind$nsk_jvmti_waitForSync 0000000180007b68     libredefclass028.obj
 0002:00002b68       $unwind$nsk_lvdisplay      0000000180007b68     libredefclass028.obj
 0002:00002b68       $unwind$_RTC_Initialize    0000000180007b68     MSVCRT:initsect.obj
 0002:00002b68       $unwind$_RTC_Terminate     0000000180007b68     MSVCRT:initsect.obj
 0002:00002b68       $unwind$?__scrt_initialize_thread_safe_statics@@YAHXZ 0000000180007b68     MSVCRT:thread_safe_statics.obj
 0002:00002b74       $unwind$nsk_complain       0000000180007b74     libredefclass028.obj
 0002:00002b74       $unwind$nsk_printf         0000000180007b74     libredefclass028.obj
 0002:00002b7c       $unwind$nsk_lvcomplain     0000000180007b7c     libredefclass028.obj
 0002:00002b94       $unwind$nsk_ltrace         0000000180007b94     libredefclass028.obj
 0002:00002b94       $unwind$__report_gsfailure 0000000180007b94     MSVCRT:gs_report.obj
 0002:00002b9c       $unwind$nsk_lvtrace        0000000180007b9c     libredefclass028.obj
 0002:00002b9c       $unwind$__raise_securityfailure 0000000180007b9c     MSVCRT:gs_report.obj
 0002:00002b9c       $unwind$__scrt_initialize_crt 0000000180007b9c     MSVCRT:utility.obj
 0002:00002b9c       $unwind$__scrt_initialize_onexit_tables 0000000180007b9c     MSVCRT:utility.obj
 0002:00002b9c       $unwind$__scrt_release_startup_lock 0000000180007b9c     MSVCRT:utility.obj
 0002:00002b9c       $unwind$__scrt_uninitialize_crt 0000000180007b9c     MSVCRT:utility.obj
 0002:00002b9c       $unwind$_onexit            0000000180007b9c     MSVCRT:utility.obj
 0002:00002ba4       $unwind$nsk_lverify        0000000180007ba4     libredefclass028.obj
 0002:00002bb4       $unwind$nsk_vprintf        0000000180007bb4     libredefclass028.obj
 0002:00002bc4       $unwind$?nsk_jni_lverify@@YAHHPEAUJNIEnv_@@HQEBDH1ZZ 0000000180007bc4     libredefclass028.obj
 0002:00002bd8       $unwind$?nsk_jni_check_exception@@YAHPEAUJNIEnv_@@QEBDH@Z 0000000180007bd8     libredefclass028.obj
 0002:00002bf4       $unwind$nsk_jvmti_parseOptions 0000000180007bf4     libredefclass028.obj
 0002:00002c10       $unwind$nsk_jvmti_createJVMTIEnv 0000000180007c10     libredefclass028.obj
 0002:00002c24       $unwind$Java_nsk_jvmti_RedefineClasses_redefclass028_isRedefinitionOccurred 0000000180007c24     libredefclass028.obj
 0002:00002c24       $unwind$Java_nsk_jvmti_RedefineClasses_redefclass028_notifyNativeAgent 0000000180007c24     libredefclass028.obj
 0002:00002c24       $unwind$Java_nsk_jvmti_unit_FollowReferences_FollowRefObjects_resetTags 0000000180007c24     libredefclass028.obj
 0002:00002c24       $unwind$addRefToVerify     0000000180007c24     libredefclass028.obj
 0002:00002c24       $unwind$nsk_jvmti_resetAgentData 0000000180007c24     libredefclass028.obj
 0002:00002c24       $unwind$nsk_jvmti_resumeSync 0000000180007c24     libredefclass028.obj
 0002:00002c24       $unwind$nsk_jvmti_setFailStatus 0000000180007c24     libredefclass028.obj
 0002:00002c24       $unwind$__scrt_initialize_default_local_stdio_options 0000000180007c24     MSVCRT:default_local_stdio_options.obj
 0002:00002c24       $unwind$?dllmain_crt_dispatch@@YAHQEAUHINSTANCE__@@KQEAX@Z 0000000180007c24     MSVCRT:dll_dllmain.obj
 0002:00002c24       $unwind$DllMain            0000000180007c24     MSVCRT:dll_dllmain_stub.obj
 0002:00002c24       $unwind$__GSHandlerCheck   0000000180007c24     MSVCRT:gshandler.obj
 0002:00002c24       $unwind$?__scrt_uninitialize_thread_safe_statics@@YAXXZ 0000000180007c24     MSVCRT:thread_safe_statics.obj
 0002:00002c24       $unwind$__scrt_acquire_startup_lock 0000000180007c24     MSVCRT:utility.obj
 0002:00002c24       $unwind$__scrt_dllmain_after_initialize_c 0000000180007c24     MSVCRT:utility.obj
 0002:00002c24       $unwind$__scrt_dllmain_before_initialize_c 0000000180007c24     MSVCRT:utility.obj
 0002:00002c24       $unwind$__scrt_dllmain_crt_thread_attach 0000000180007c24     MSVCRT:utility.obj
 0002:00002c24       $unwind$__scrt_dllmain_crt_thread_detach 0000000180007c24     MSVCRT:utility.obj
 0002:00002c24       $unwind$__scrt_dllmain_uninitialize_c 0000000180007c24     MSVCRT:utility.obj
 0002:00002c24       $unwind$__scrt_dllmain_uninitialize_critical 0000000180007c24     MSVCRT:utility.obj
 0002:00002c24       $unwind$atexit             0000000180007c24     MSVCRT:utility.obj
 0002:00002c2c       $unwind$nsk_jvmti_enableEvents 0000000180007c2c     libredefclass028.obj
 0002:00002c44       $unwind$nsk_jvmti_lverify  0000000180007c44     libredefclass028.obj
 0002:00002c58       $unwind$exitOnError        0000000180007c58     libredefclass028.obj
 0002:00002c68       $unwind$check_option       0000000180007c68     libredefclass028.obj
 0002:00002c68       $unwind$_DllMainCRTStartup 0000000180007c68     MSVCRT:dll_dllmain.obj
 0002:00002c78       $unwind$Java_nsk_share_jvmti_ArgumentHandler_getAgentOptionsString 0000000180007c78     libredefclass028.obj
 0002:00002c8c       $unwind$Java_nsk_jvmti_unit_FollowReferences_FollowRefObjects_getTag 0000000180007c8c     libredefclass028.obj
 0002:00002c8c       $unwind$Java_nsk_share_jvmti_DebugeeClass_checkStatus 0000000180007c8c     libredefclass028.obj
 0002:00002c8c       $unwind$agentThreadWrapper 0000000180007c8c     libredefclass028.obj
 0002:00002c9c       $unwind$startAgentThreadWrapper 0000000180007c9c     libredefclass028.obj
 0002:00002cb8       $unwind$syncDebuggeeStatus 0000000180007cb8     libredefclass028.obj
 0002:00002cb8       $unwind$__scrt_dllmain_exception_filter 0000000180007cb8     MSVCRT:utility.obj
 0002:00002ccc       $unwind$Java_nsk_share_jvmti_DebugeeClass_resetAgentData 0000000180007ccc     libredefclass028.obj
 0002:00002cd4       $unwind$MA_checkStatus     0000000180007cd4     libredefclass028.obj
 0002:00002ce8       $unwind$Java_nsk_jvmti_unit_FollowReferences_FollowRefObjects_setTag 0000000180007ce8     libredefclass028.obj
 0002:00002d00       $unwind$Java_nsk_jvmti_unit_FollowReferences_FollowRefObjects_addRefToVerify 0000000180007d00     libredefclass028.obj
 0002:00002d1c       $unwind$Agent_Initialize   0000000180007d1c     libredefclass028.obj
 0002:00002d40       $unwind$Java_nsk_jvmti_RedefineClasses_redefclass028_storeClassBytes 0000000180007d40     libredefclass028.obj
 0002:00002d4c       $unwind$CompiledMethodLoad 0000000180007d4c     libredefclass028.obj
 0002:00002d64       $unwind$CompiledMethodUnload 0000000180007d64     libredefclass028.obj
 0002:00002d74       $unwind$agentProc          0000000180007d74     libredefclass028.obj
 0002:00002d8c       $unwind$capture_previous_context 0000000180007d8c     MSVCRT:gs_report.obj
 0002:00002d98       $unwind$__GSHandlerCheckCommon 0000000180007d98     MSVCRT:gshandler.obj
 0002:00002da0       $xdatasym                  0000000180007da0     MSVCRT:amdsecgs.obj
 0002:00002da4       $unwind$?dllmain_crt_process_attach@@YAHQEAUHINSTANCE__@@QEAX@Z 0000000180007da4     MSVCRT:dll_dllmain.obj
 0002:00002de0       $unwind$?fin$0@?0??dllmain_crt_process_attach@@YAHQEAUHINSTANCE__@@QEAX@Z@4HA 0000000180007de0     MSVCRT:dll_dllmain.obj
 0002:00002de0       $unwind$?fin$0@?0??dllmain_crt_process_detach@@YAH_N@Z@4HA 0000000180007de0     MSVCRT:dll_dllmain.obj
 0002:00002de0       $unwind$?fin$1@?0??dllmain_crt_process_detach@@YAH_N@Z@4HA 0000000180007de0     MSVCRT:dll_dllmain.obj
 0002:00002de8       $unwind$?dllmain_crt_process_detach@@YAH_N@Z 0000000180007de8     MSVCRT:dll_dllmain.obj
 0002:00002e3c       $unwind$?dllmain_dispatch@@YAHQEAUHINSTANCE__@@KQEAX@Z 0000000180007e3c     MSVCRT:dll_dllmain.obj
 0002:00002e64       $unwind$?filt$0@?0??dllmain_dispatch@@YAHQEAUHINSTANCE__@@KQEAX@Z@4HA 0000000180007e64     MSVCRT:dll_dllmain.obj
 0002:00002e6c       $unwind$__scrt_is_nonwritable_in_current_image 0000000180007e6c     MSVCRT:utility.obj
 0002:00002e8c       $unwind$__scrt_is_nonwritable_in_current_image$filt$0 0000000180007e8c     MSVCRT:utility.obj
 0002:00002e94       $unwind$__scrt_fastfail    0000000180007e94     MSVCRT:utility_desktop.obj
 0002:00002ea4       $unwind$__security_init_cookie 0000000180007ea4     MSVCRT:gs_support.obj
 0002:00002eb0       $unwind$__isa_available_init 0000000180007eb0     MSVCRT:cpu_disp.obj
 0002:00002ec0       $xdatasym                  0000000180007ec0     MSVCRT:guard_dispatch.obj
 0002:00002ec8       $xdatasym                  0000000180007ec8     MSVCRT:guard_xfg_dispatch.obj
 0002:00002ed0       .edata                     0000000180007ed0     redefclass028.exp
 0002:00002ef8       rgpv                       0000000180007ef8     redefclass028.exp
 0002:00002f40       rgszName                   0000000180007f40     redefclass028.exp
 0002:00002f88       rgwOrd                     0000000180007f88     redefclass028.exp
 0002:00002fac       szName                     0000000180007fac     redefclass028.exp
 0002:00002fbe       $N00001                    0000000180007fbe     redefclass028.exp
 0002:00002fcd       $N00002                    0000000180007fcd     redefclass028.exp
 0002:00002fda       $N00003                    0000000180007fda     redefclass028.exp
 0002:00002fef       $N00004                    0000000180007fef     redefclass028.exp
 0002:00003033       $N00005                    0000000180008033     redefclass028.exp
 0002:00003072       $N00006                    0000000180008072     redefclass028.exp
 0002:000030af       $N00007                    00000001800080af     redefclass028.exp
 0002:000030f4       $N00008                    00000001800080f4     redefclass028.exp
 0002:00003131       $N00009                    0000000180008131     redefclass028.exp
 0002:00003179       $N00010                    0000000180008179     redefclass028.exp
 0002:000031b9       $N00011                    00000001800081b9     redefclass028.exp
 0002:000031f6       $N00012                    00000001800081f6     redefclass028.exp
 0002:00003231       $N00013                    0000000180008231     redefclass028.exp
 0002:0000325f       $N00014                    000000018000825f     redefclass028.exp
 0002:00003290       $N00015                    0000000180008290     redefclass028.exp
 0002:000032bf       $N00016                    00000001800082bf     redefclass028.exp
 0002:000032ee       $N00017                    00000001800082ee     redefclass028.exp
 0002:00003323       $N00018                    0000000180008323     redefclass028.exp
 0002:0000379a       .idata$6                   000000018000879a     kernel32:KERNEL32.dll
 0002:000037fe       .idata$6                   00000001800087fe     vcruntime:VCRUNTIME140.dll
 0002:00003990       .idata$6                   0000000180008990     ucrt:api-ms-win-crt-heap-l1-1-0.dll
 0002:000039b0       .idata$6                   00000001800089b0     ucrt:api-ms-win-crt-runtime-l1-1-0.dll
 0002:000039d2       .idata$6                   00000001800089d2     ucrt:api-ms-win-crt-convert-l1-1-0.dll
 0002:000039f4       .idata$6                   00000001800089f4     ucrt:api-ms-win-crt-stdio-l1-1-0.dll
 0002:00003a14       .idata$6                   0000000180008a14     ucrt:api-ms-win-crt-string-l1-1-0.dll
 0003:00000000       ?codeAttributeName@@3PEBDEB 0000000180009000     libredefclass028.obj
 0003:00000008       ?lineNumberAttributeName@@3PEBDEB 0000000180009008     libredefclass028.obj
 0003:00000010       ?localVarAttributeName@@3PEBDEB 0000000180009010     libredefclass028.obj
 0003:00000018       ?localVarTypeAttributeName@@3PEBDEB 0000000180009018     libredefclass028.obj
 0003:00000020       ?stackMapAttributeName@@3PEBDEB 0000000180009020     libredefclass028.obj
 0003:00000028       ?callBytes@@3PAEA          0000000180009028     libredefclass028.obj
 0003:0000002c       ?allocBytes@@3PAEA         000000018000902c     libredefclass028.obj
 0003:00000030       expHSMethod                0000000180009030     libredefclass028.obj
 0003:00000038       expHSSignature             0000000180009038     libredefclass028.obj
 0003:00000040       eventsList                 0000000180009040     libredefclass028.obj
 0003:0001aae4       redefineAttempted          0000000180023ae4     libredefclass028.obj
 0003:0001aae8       nsk_context                0000000180023ae8     libredefclass028.obj
 0003:0001aaf4       redefineSucceed            0000000180023af4     libredefclass028.obj
 0003:0001aaf8       agentFailed                0000000180023af8     libredefclass028.obj
 0003:0001aafc       currentAgentStatus         0000000180023afc     libredefclass028.obj
 0003:0001ab00       context                    0000000180023b00     libredefclass028.obj
 0003:0001abb8       agentThread                0000000180023bb8     libredefclass028.obj
 0003:0001abc0       agentThreadProc            0000000180023bc0     libredefclass028.obj
 0003:0001abc8       agentThreadArg             0000000180023bc8     libredefclass028.obj
 0003:0001abd0       agent_data                 0000000180023bd0     libredefclass028.obj
 0003:0001abe0       jvmti_env                  0000000180023be0     libredefclass028.obj
 0003:0001abe8       jvm                        0000000180023be8     libredefclass028.obj
 0003:0001abf0       jni_env                    0000000180023bf0     libredefclass028.obj
 0003:0001abf8       checkStatus_func           0000000180023bf8     libredefclass028.obj
 0003:0001ac00       ?codeAttributeIndex@@3GA   0000000180023c00     libredefclass028.obj
 0003:0001ac04       ?lineNumberAttributeIndex@@3GA 0000000180023c04     libredefclass028.obj
 0003:0001ac08       ?localVarAttributeIndex@@3GA 0000000180023c08     libredefclass028.obj
 0003:0001ac0c       ?localVarTypeAttributeIndex@@3GA 0000000180023c0c     libredefclass028.obj
 0003:0001ac10       ?stackMapAttributeIndex@@3GA 0000000180023c10     libredefclass028.obj
 0003:0001ac14       ?stackFrameOffset@@3GA     0000000180023c14     libredefclass028.obj
 0003:0001ac18       ?mode@@3HA                 0000000180023c18     libredefclass028.obj
 0003:0001ac1c       ?constantPoolSize@@3GA     0000000180023c1c     libredefclass028.obj
 0003:0001ac20       ?orig@@3PEBEEB             0000000180023c20     libredefclass028.obj
 0003:0001ac28       ?gen@@3PEAEEA              0000000180023c28     libredefclass028.obj
 0003:0001ac30       ?inputPos@@3PEAEEA         0000000180023c30     libredefclass028.obj
 0003:0001ac38       ?endPos@@3PEBEEB           0000000180023c38     libredefclass028.obj
 0003:0001ac40       ?genPos@@3PEAEEA           0000000180023c40     libredefclass028.obj
 0003:0001ac48       ?markPos@@3PEAEEA          0000000180023c48     libredefclass028.obj
 0003:0001ac50       ?constantPool@@3PEAPEADEA  0000000180023c50     libredefclass028.obj
 0003:0001ac58       ?constantPoolCount@@3GA    0000000180023c58     libredefclass028.obj
 0003:0001ac5c       ?zeroBytes@@3PAEA          0000000180023c5c     libredefclass028.obj
 0003:0001ac60       ?codeLength@@3IA           0000000180023c60     libredefclass028.obj
 0003:0001ac64       fire                       0000000180023c64     libredefclass028.obj
 0003:0001ac68       ?map@@3PEAIEA              0000000180023c68     libredefclass028.obj
 0003:0001ac70       ?widening@@3PEACEA         0000000180023c70     libredefclass028.obj
 0003:0001ac78       jvmti                      0000000180023c78     libredefclass028.obj
 0003:0001ac80       timeout                    0000000180023c80     libredefclass028.obj
 0003:0001ac88       hsMethodID                 0000000180023c88     libredefclass028.obj
 0003:0001ac90       enteredHotMethod           0000000180023c90     libredefclass028.obj
 0003:0001ac94       bytesCount                 0000000180023c94     libredefclass028.obj
 0003:0001ac98       clsBytes                   0000000180023c98     libredefclass028.obj
 0003:0001acb0       GS_ExceptionRecord         0000000180023cb0     MSVCRT:gs_report.obj
 0003:0001ad50       GS_ContextRecord           0000000180023d50     MSVCRT:gs_report.obj
 0003:0001b220       ?g_tss_cv@@3U_RTL_CONDITION_VARIABLE@@A 0000000180024220     MSVCRT:thread_safe_statics.obj
 0003:0001b228       ?g_tss_event@@3PEAXEA      0000000180024228     MSVCRT:thread_safe_statics.obj
 0003:0001b230       ?g_tss_mutex@@3U_RTL_CRITICAL_SECTION@@A 0000000180024230     MSVCRT:thread_safe_statics.obj
 0003:0001b258       ?g_sleep_condition_variable_cs@@3P6AHPEAU_RTL_CONDITION_VARIABLE@@PEAU_RTL_CRITICAL_SECTION@@K@ZEA 0000000180024258     MSVCRT:thread_safe_statics.obj
 0003:0001b260       ?g_wake_all_condition_variable@@3P6AXPEAU_RTL_CONDITION_VARIABLE@@@ZEA 0000000180024260     MSVCRT:thread_safe_statics.obj
 0003:0001b26c       ?__proc_attached@@3HA      000000018002426c     MSVCRT:dll_dllmain.obj
 0003:0001b280       ?is_initialized_as_dll@@3_NA 0000000180024280     MSVCRT:utility.obj
 0003:0001b281       ?module_local_atexit_table_initialized@@3_NA 0000000180024281     MSVCRT:utility.obj
 0003:0001b288       ?module_local_atexit_table@@3U_onexit_table_t@@A 0000000180024288     MSVCRT:utility.obj
 0003:0001b2a0       ?module_local_at_quick_exit_table@@3U_onexit_table_t@@A 00000001800242a0     MSVCRT:utility.obj
